:100000004BC0FEC034C163C062C061C061C051C298
:100010005EC09AC15CC029C24AC112C450C48EC419
:10002000BEC4FDC4A0C5D3C577C633C832C8F6C6A2
:10003000446D697472792050756B686F76277320F0
:1000400070726962616D62617320776172652E0002
:1000500050446D69747279406D61696C2E72752CB3
:10006000206963712035353637363135332E004EF1
:100070006F7620323720546875727364617920324C
:100080003030370046616E74616B75204162757067
:10009000616261203234000011241FBECFE5D2E03E
:1000A000DEBFCDBF10E0A0E6B0E0E8E0FAE103C0BB
:1000B000C89531960D92A036B107D1F710E0A0E6B1
:1000C000B0E001C01D92A43EB107E1F7FAC298CF9B
:1000D0001F920F920FB60F9211248F939F93AF939D
:1000E000BF9386EF92EC9DBD8CBD8091D500909121
:1000F000D6009093A2008093A1001092D600109297
:10010000D50080916000813029F58091D9009091CF
:10011000DA0090937200809371008091A300909117
:10012000A40090936300809362008091D700909127
:10013000D80090936500809364001092A400109200
:10014000A3001092DA001092D9001092D8001092F9
:10015000D70024C08091D2009091D3009093720078
:10016000809371008091C8009091C90090936300C2
:10017000809362008091CA009091CB0090936500BB
:10018000809364001092C9001092C8001092D300AE
:100190001092D2001092CB001092CA0080916000A1
:1001A0008F5F8170809360008091690090916A00F8
:1001B000A0916B00B0916C000196A11DB11D8093C0
:1001C000690090936A00A0936B00B0936C008091DB
:1001D0009D0088232CF48091D4008F5F8093D400FD
:1001E0008091D100803118F481508093D100BF916B
:1001F000AF919F918F910F900FBE0F901F90189508
:100200001F920F920FB60F9211248F939F93AF936B
:10021000BF938091A3009091A40001969093A400B5
:100220008093A3008091C8009091C900019690939B
:10023000C9008093C80080916D0090916E00A091DC
:100240006F00B09170000196A11DB11D80936D00EB
:1002500090936E00A0936F00B0937000BF91AF9128
:100260009F918F910F900FBE0F901F9018951F9226
:100270000F920FB60F9211248F939F938091D70006
:100280009091D80001969093D8008093D7008091E8
:10029000CA009091CB0001969093CB008093CA0046
:1002A0009F918F910F900FBE0F901F9018951F92E6
:1002B0000F920FB60F9211248F939F93AF93BF931A
:1002C0008091D9009091DA0001969093DA008093A2
:1002D000D9008091D2009091D30001969093D300E1
:1002E0008093D200B69914C08091730090917400ED
:1002F000A0917500B09176000196A11DB11D80936B
:10030000730090937400A0937500B093760013C0AF
:1003100080917B0090917C00A0917D00B0917E0047
:100320000196A11DB11D80937B0090937C00A0934A
:100330007D00B0937E00BF91AF919F918F910F9000
:100340000FBE0F901F9018951F920F920FB60F922D
:1003500011242F938F939F93EF93FF932CB1809150
:10036000CE008823A1F0E091CC00F091CD00208355
:100370008091CC009091CD0001969093CD00809318
:10038000CC008091CE0081508093CE0064C0822F3B
:100390009927823F9105C1F1833F91053CF4803F4D
:1003A0009105E1F0813F910521F14FC0843F910516
:1003B00009F440C0843F910594F18E3F910509F006
:1003C00044C082E690E09093CD008093CC00579893
:1003D000569A81E48093CE008CB93DC084E080932E
:1003E000CE008CB983E890E09093CD008093CC0050
:1003F00032C084E08093CE008CB987E890E090937F
:10040000CD008093CC0027C084E08093CE008CB9CF
:100410008BE890E09093CD008093CC001CC084E0EA
:100420008093CE008CB98FE890E09093CD008093BC
:10043000CC0011C084E08093CE008CB983E990E0B9
:100440009093CD008093CC0006C0822F805D8B30CE
:1004500010F42093A000FF91EF919F918F912F9125
:100460000F900FBE0F901F9018951F920F920FB60E
:100470000F9211248F93EF93FF93E091CC00F091B2
:10048000CD008191F093CD00E093CC008CB98091A8
:10049000CE0081508093CE00882319F48CB15698F9
:1004A000579AFF91EF918F910F900FBE0F901F9071
:1004B00018951F920F920FB60F9211242F933F930E
:1004C0004F935F938F939F93EF93FF938EEC82BF35
:1004D00015BA8BB3807F8BBB50916100252F3327DA
:1004E00081E090E0022E02C0880F991F0A94E2F783
:1004F0004BB3842B8BBB932F822F820F931FF92F2B
:10050000E82FE452FF4F80819181F92FE82FEB55BE
:10051000FF4F808185BB852F8F5F83708093610043
:10052000D89B2DC0C4992BC08091CF009091D00052
:10053000880F991F9093D0008093CF00B59B05C082
:1005400001969093D0008093CF008091DB008F5F65
:100550008093DB00883099F4C49A209166008091E2
:10056000CF009091D000820F911D96958795809332
:1005700066001092D0001092CF001092DB00DA9942
:10058000C498809199008F5F80939900859B06C0E5
:10059000882334F480E88093990002C01092990077
:1005A00080919A008F5F80939A00869B06C0882373
:1005B00034F480E880939A0002C010929A008091EF
:1005C0009B008F5F80939B00879B06C0882334F439
:1005D00080E880939B0002C010929B0080919C0059
:1005E000982F9F5F90939C0080919D008F5F8093D8
:1005F0009D00849917C010929D00903149F480911C
:10060000D400823028F48091A0008F5F8093A000F6
:1006100080919C008823D4F480E880939C00109201
:10062000D40014C010929C0080919D00803139F458
:100630008091D100803119F08FE08093D1008091BA
:100640009D0088231CF480E880939D0080919E008B
:100650008F5F80939E00B09B06C0882334F480E8AF
:1006600080939E0002C010929E00B69B04C080E85A
:1006700080939F0002C010929F00FF91EF919F9185
:100680008F915F914F913F912F910F900FBE0F90DF
:100690001F9018951BBA9FEF9ABB8FE488BB80E927
:1006A00087BBC798C49A15BA94BB82E081BB8CE023
:1006B00082BB089589E189B91BB888E98AB98CB1F0
:1006C0000895CFE5D2E0DEBFCDBFE4DFF3DFE5EA9A
:1006D000F0E0A1E4B0E081E290E021E08030920718
:1006E00011F45DD902C0182E5AD9E2E6F0E0A0E07C
:1006F000B0E081E490E021E08030920711F44FD91E
:1007000002C0182E4CD91092D3001092D200109231
:10071000DA001092D9001092CE001092CB00109205
:10072000CA001092D8001092D7001092C9001092FF
:10073000C8001092A4001092A3001092D60010924C
:10074000D5001092D0001092CF001092D4001092D9
:10075000DB001092720010927100109265001092EE
:100760006400109263001092620010926600809103
:10077000A0008F5C8C3018F08FEC8093A0008EEC82
:1007800082BF24E023BF86EF92EC9DBD8CBD2EBDC1
:1007900082E889BF85B78F6085BF80EC8BBF8AE018
:1007A00088B9789480E18093D100209162003091E3
:1007B000630080916700909168008217930720F48E
:1007C00030936800209367008091D400823039F51F
:1007D00010926D0010926E0010926F0010927000D7
:1007E0001092690010926A0010926B0010926C00D7
:1007F00010927B0010927C0010927D0010927E007F
:10080000109273001092740010927500109276008E
:1008100010926800109267008F5F8093D400C0E050
:100820008091A0009927AA27BB27F92FE82FE05D28
:10083000F040EB30F10508F02CC4E35FFF4F099462
:100840000091620010916300802F912FAA2797FDDD
:10085000A095BA2F682F792F8A2F9B2FD8D71123D5
:100860002CF420E030E040E857E42CD720918300BE
:1008700030918400409185005091860042D8B92F74
:10088000A82F972F862F20E030E040E951E4682F11
:10089000792F8A2F9B2F35D8B92FA82F972F862FE6
:1008A000682F792F8A2F9B2F95D7B92FA82F972F95
:1008B000862F9093C7008093C60001E021C6009167
:1008C000640010916500802F912FAA2797FDA095B5
:1008D000BA2F682F792F8A2F9B2F99D711232CF4A9
:1008E00020E030E040E857E4EDD6209187003091D9
:1008F00088004091890050918A0003D8B92FA82F11
:10090000972F862F20E030E040E05FE3682F792FBB
:100910008A2F9B2FF6D7B92FA82F972F862F682FB6
:10092000792F8A2F9B2F56D7B92FA82F972F862F35
:100930009093C7008093C60000E0E2C51091660066
:10094000812F992787FD9095A92FB92F682F792F8F
:100950008A2F9B2F5CD711232CF420E030E040E855
:1009600053E4B0D6209193003091940040919500CB
:1009700050919600C6D7B92FA82F972F862F682F92
:10098000792F8A2F9B2F26D7B92FA82F972F862F05
:100990009093C7008093C600C8E101E0B1C5009103
:1009A000670010916800802F912FAA2797FDA095CE
:1009B000BA2F682F792F8A2F9B2F29D711232CF438
:1009C00020E030E040E857E47DD62091830030916C
:1009D0008400409185005091860093D7B92FA82FAD
:1009E000972F862F26E636E646EE5FE3682F792FAF
:1009F0008A2F9B2F86D7B92FA82F972F862F682F46
:100A0000792F8A2F9B2FE6D6B92FA82F972F862FC5
:100A10009093C7008093C6000FEFC9E171C5809124
:100A2000690090916A00A0916B00B0916C000097F2
:100A3000A105B10529F41092C7001092C60090C01C
:100A400060916D0070916E0080916F0090917000C8
:100A5000992314F0DCD622C080916D0090916E0035
:100A6000A0916F00B0917000282F392F4A2F5B2F73
:100A70002170307040705070B695A7959795879506
:100A8000282B392B4A2B5B2B952F842F732F622F0A
:100A9000BED6262F372F482F592F14D620918300EA
:100AA0003091840040918500509186002AD7B92F5B
:100AB000A82F972F862F26E636E646E650E4682FC5
:100AC000792F8A2F9B2F1DD7E62EF72E082F192F4F
:100AD0006091690070916A0080916B0090916C0048
:100AE000992314F094D622C08091690090916A00F5
:100AF000A0916B00B0916C00282F392F4A2F5B2FEB
:100B00002170307040705070B695A7959795879575
:100B1000282B392B4A2B5B2B952F842F732F622F79
:100B200076D6262F372F482F592FCCD5262F372F63
:100B3000482F592F912F802F7F2D6E2D05D6B92F3D
:100B4000A82F972F862F682F792F8A2F9B2F42D679
:100B5000B92FA82F972F862F9093C7008093C60098
:100B60000FEFCAE1CDC48091690090916A006CE3F7
:100B700070E033D77093C7006093C6006057774129
:100B800020F110927B0010927C0010927D00109258
:100B90007E001092730010927400109275001092F3
:100BA00076001092690010926A0010926B00109209
:100BB0006C0010926D0010926E0010926F001092F7
:100BC00070001092C7001092C60002E099C46091B4
:100BD0006D0070916E0080916F009091700099236C
:100BE00034F015D6C62ED72EE82EF92E26C08091C9
:100BF0006D0090916E00A0916F00B0917000282F51
:100C0000392F4A2F5B2F2170307040705070B6958D
:100C1000A79597958795282B392B4A2B5B2B952FDA
:100C2000842F732F622FF3D5262F372F482F592F5C
:100C300049D5C62ED72EE82EF92E2091830030916B
:100C4000840040918500509186009F2D8E2D7D2D32
:100C50006C2D57D6C62ED72EE82EF92E20E030E484
:100C60004CE156E4DED588237CF49F2D8E2D7D2D1E
:100C70006C2DB0D5B92FA82F972F862F9093C70032
:100C80008093C60003E01BC020E030E04AE754E454
:100C90009F2D8E2D7D2D6C2D57D5B92FA82F972FD9
:100CA000862F682F792F8A2F9B2F94D5B92FA82FA5
:100CB000972F862F9093C7008093C60000E0809105
:100CC000C6009091C7008051974208F419C4109251
:100CD0007B0010927C0010927D0010927E0010929A
:100CE00073001092740010927500109276001092AA
:100CF000690010926A0010926B0010926C001092C2
:100D00006D0010926E0010926F00109270001092A1
:100D1000C7001092C600F4C380919F008823F1F5AC
:100D20000091710010917200802F912FAA2797FDDA
:100D3000A095BA2F682F792F8A2F9B2F68D5112362
:100D40002CF420E030E040E857E4BCD420918B0044
:100D500030918C0040918D0050918E00D2D5B92FEA
:100D6000A82F972F862F20E030E040EA50E4682F2C
:100D7000792F8A2F9B2FC5D5B92FA82F972F862F74
:100D8000682F792F8A2F9B2F25D5B92FA82F972F22
:100D9000862F9093C7008093C6003DC000917100DC
:100DA00010917200802F912FAA2797FDA095BA2F3E
:100DB000682F792F8A2F9B2F2AD511232CF420E01E
:100DC00030E040E857E47ED420918F0030919000CD
:100DD000409191005091920094D5B92FA82F972F50
:100DE000862F20E030E040EA50E4682F792F8A2FE8
:100DF0009B2F87D5B92FA82F972F862F682F792F54
:100E00008A2F9B2FE7D4B92FA82F972F862F909347
:100E1000C7008093C60002E0CCE172C3CAE08091B3
:100E20009F00882309F049C060917300709174009D
:100E30008091750090917600992334F0E8D4C62E05
:100E4000D72EE82EF92E27C08FE990E0F92FE82F52
:100E5000BC972081318142815381B52FA42F932FDC
:100E6000822F81709070A070B0705695479537951D
:100E70002795822B932BA42BB52B682F792F8A2FA4
:100E80009B2FC5D4262F372F482F592F1BD4C62E62
:100E9000D72EE82EF92E20918B0030918C004091B6
:100EA0008D0050918E009F2D8E2D7D2D6C2D29D57E
:100EB000C62ED72EE82EF92E48C060917B00709187
:100EC0007C0080917D0090917E00992334F09FD426
:100ED000C62ED72EE82EF92E26C080917B00909149
:100EE0007C00A0917D00B0917E00282F392F4A2FE1
:100EF0005B2F2170307040705070B695A795979514
:100F00008795282B392B4A2B5B2B952F842F732FFA
:100F1000622F7DD4262F372F482F592FD3D3C62E9B
:100F2000D72EE82EF92E20918F003091900040911D
:100F30009100509192009F2D8E2D7D2D6C2DE1D42E
:100F4000C62ED72EE82EF92ECF5F20E030E44CE1FC
:100F500056E49F2D8E2D7D2D6C2D63D488237CF43B
:100F600003E020E030E040E251E49F2D8E2D7D2D06
:100F70006C2DEAD3C62ED72EE82EF92E42C020E0E3
:100F800030E543EC57E49F2D8E2D7D2D6C2D49D4FB
:100F900088237CF402E020E030E048EC52E49F2D0E
:100FA0008E2D7D2D6C2DD0D3C62ED72EE82EF92E6A
:100FB00028C020E034E244E759E49F2D8E2D7D2D9A
:100FC0006C2D2FD488237CF401E020E030E04AE748
:100FD00054E49F2D8E2D7D2D6C2DB6D3C62ED72E8D
:100FE000E82EF92E0EC000E020E030E44CE156E49B
:100FF0009F2D8E2D7D2D6C2DA7D3C62ED72EE82E9E
:10100000F92E20E030E040E05FE39F2D8E2D7D2D16
:101010006C2D58D3B92FA82F972F862F682F792F93
:101020008A2F9B2FD7D3B92FA82F972F862F282F02
:10103000392F9093C7008093C600002309F060C247
:101040002051374208F45CC210927B0010927C0061
:1010500010927D0010927E00109273001092740026
:1010600010927500109276001092690010926A003A
:1010700010926B0010926C0010926D0010926E0036
:1010800010926F00109270001092C7001092C6006C
:1010900037C28091A0009927883D910529F0893DAC
:1010A000910509F422C1ADC1CDE180917300909109
:1010B0007400A0917500B09176000097A105B1056C
:1010C00021F480919F00882381F080917B00909192
:1010D0007C00A0917D00B0917E000097A105B10534
:1010E00079F480919F00803859F40F2EF0E0CF2ED4
:1010F000F0E0DF2EF0E0EF2EF0E0FF2EF02D8EC1BD
:1011000080916D0090916E00A0916F00B091700081
:101110000097A105B10559F40F2EF0E0CF2EF0E0B5
:10112000DF2EFAE7EF2EF4E4FF2EF02D77C1809149
:101130009F00882309F049C060917300709174008A
:101140008091750090917600992334F060D3C62E7B
:10115000D72EE82EF92E27C08FE990E0F92FE82F3F
:10116000BC972081318142815381B52FA42F932FC9
:10117000822F81709070A070B0705695479537950A
:101180002795822B932BA42BB52B682F792F8A2F91
:101190009B2F3DD3262F372F482F592F93D2C62E62
:1011A000D72EE82EF92E20918B0030918C004091A3
:1011B0008D0050918E009F2D8E2D7D2D6C2DA1D3F5
:1011C000C62ED72EE82EF92E47C060917B00709175
:1011D0007C0080917D0090917E00992334F017D39C
:1011E000C62ED72EE82EF92E26C080917B00909136
:1011F0007C00A0917D00B0917E00282F392F4A2FCE
:101200005B2F2170307040705070B695A795979500
:101210008795282B392B4A2B5B2B952F842F732FE7
:10122000622FF5D2262F372F482F592F4BD2C62E9B
:10123000D72EE82EF92E20918F003091900040910A
:101240009100509192009F2D8E2D7D2D6C2D59D3A4
:10125000C62ED72EE82EF92E60916D0070916E008B
:1012600080916F0090917000992314F0D0D222C029
:1012700080916D0090916E00A0916F00B091700010
:10128000282F392F4A2F5B2F2170307040705070FB
:10129000B695A79597958795282B392B4A2B5B2BCD
:1012A000952F842F732F622FB2D2262F372F482FDE
:1012B000592F08D2209183003091840040918500FD
:1012C000509186001ED3B92FA82F972F862F282F35
:1012D000392F4A2F5B2F9F2D8E2D7D2D6C2D34D2D3
:1012E000C62ED72EE82EF92E99C0CEE1809171003E
:1012F00090917200892B59F40F2EF0E0CF2EF0E080
:10130000DF2EF0E0EF2EF0E0FF2EF02D87C0809171
:10131000620090916300892B59F40F2EF0E0CF2EDC
:10132000F0E0DF2EFAE7EF2EF4E4FF2EF02D76C08A
:1013300080919F00882349F4C0908B00D0908C004E
:10134000E0908D00F0908E0008C0C0908F00D0908B
:101350009000E0909100F090920000917100109147
:101360007200802F912FAA2797FDA095BA2F682F82
:10137000792F8A2F9B2F4BD211232CF420E030E0C1
:1013800040E857E49FD1262F372F482F592F9F2D04
:101390008E2D7D2D6C2DB5D2C62ED72EE82EF92E92
:1013A0000091620010916300802F912FAA2797FD72
:1013B000A095BA2F682F792F8A2F9B2F28D211231F
:1013C0002CF420E030E040E857E47CD12091830009
:1013D00030918400409185005091860092D2B92FBF
:1013E000A82F972F862F282F392F4A2F5B2F9F2D1D
:1013F0008E2D7D2D6C2DA8D1C62ED72EE82EF92E40
:101400000DC080ED8093A0000F2EF0E0CF2EF0E015
:10141000DF2EF0E0EF2EF0E0FF2EF02D20E030E0A8
:1014200040E85FE39F2D8E2D7D2D6C2DFAD1882312
:101430007CF402E020E030E04AE754E49F2D8E2D5A
:101440007D2D6C2D5ED2C62ED72EE82EF92E3EC0F5
:1014500020E030E040E251E49F2D8E2D7D2D6C2D5B
:10146000E0D188237CF401E020E030E048EC52E455
:101470009F2D8E2D7D2D6C2D44D2C62ED72EE82E7D
:10148000F92E24C000E020E030E048EC52E49F2D2B
:101490008E2D7D2D6C2DC5D1882374F420E030E095
:1014A00040E251E49F2D8E2D7D2D6C2D2AD2C62E2B
:1014B000D72EE82EF92E0AC00F2EF0E0CF2EF0EC3A
:1014C000DF2EF9E7EF2EF4E4FF2EF02D20E030E0E0
:1014D00040E05FE39F2D8E2D7D2D6C2DF3D0B92F35
:1014E000A82F972F862F682F792F8A2F9B2F72D1A5
:1014F000B92FA82F972F862F9093C7008093C600EF
:101500008091C6009091C70060E177E266D2282FF3
:10151000392F9093C7008093C6008091A000853D2D
:1015200009F5CC2331F4932F822F68E572E055D270
:10153000C62F8091C6009091C70068E572E04DD239
:10154000282F392FECE3F0E06E2F7F2F46D2162F95
:10155000932F822F6E2F7F2F40D29093C7008093BE
:10156000C60022C0CC2341F48091C6009091C700F0
:1015700068EE73E032D2C62F8091C6009091C7000A
:1015800068EE73E02AD2282F392FE4E6F0E06E2FC0
:101590007F2F23D2162F932F822F6E2F7F2F1DD2B6
:1015A0009093C7008093C6002091C6003091C70079
:1015B000EAE0F0E0932F822F6E2F7F2F0ED2462F7E
:1015C000932F822F6E2F7F2F08D2202F3327213089
:1015D000310579F0223031051CF4232B41F00EC087
:1015E0002230310541F02330310539F007C0845FE6
:1015F00005C0445F03C0145F01C0C45FCC2339F44D
:10160000C0E2112321F41C2F442309F44C2FC831CC
:1016100030F0112321F410E2442309F4412F9927DB
:101620009093DD008093DC00842F99279093DF0056
:101630008093DE00812F99279093E1008093E00052
:101640008C2F99279093E3008093E2008091D5003E
:101650009091D60001969093D6008093D500B199D1
:1016600009C0B99AC19A8091D100803119F48FE0F4
:101670008093D1008091D100882309F096C8B99851
:10168000C19AB1998FC8F8941EBC8EB583BF83B739
:1016900085BB85B38BBBB99AC19AE2E6F0E0A0E0C6
:1016A000B0E081E490E021E08030920711F47CD139
:1016B00002C0182E79D1C198889580E090E000C0D2
:1016C000A2C15058192EEFD001D0D2C0BA1762076C
:1016D000730784079507B1F188F40EF410940B2E6C
:1016E000BA2FA02D062E622F202D072E732F302DFE
:1016F000082E842F402D092E952F502DFF2755237E
:10170000B9F0591B49F0573E98F046953795279503
:10171000A795F0405395C9F776F0BA0F621F731F73
:10172000841F30F4879577956795B795F04093952A
:1017300017FA0F2E0895BF1BBB27BA0B620B730B52
:10174000840BF6CFDEF6DBC0AED001D091C05523BE
:1017500059F0992369F09F575F57951B33F442F472
:10176000903811F4915805C09BC091589F3F09F4DF
:10177000C6C0BB27112462177307840730F4660FB5
:10178000771F881FBB1F915098F311D00F920FD075
:101790000F920DD0A0E82617370748071B0609F05F
:1017A000A048BA2F602D7F918F9100240895A0E862
:1017B0000024621773078407B10528F0621B730BBE
:1017C000840BB1090A2A660F771F881FBB1FA695D5
:1017D00081F7089597FB73D09F3738F0FEE9F91B26
:1017E000982F872F762F6B2F05C086C096958795EB
:1017F00077956795F150D0F73EF490958095709568
:1018000061957F4F8F4F9F4F0895E89403C097FBDA
:101810000EF4F3DFB62F672F782F892F9EE900246F
:1018200027C00ED05EF004C00BD026F001C008D057
:1018300019F020F48FEF089580E0089581E0089575
:1018400097FB092E052600F8689430D0E89407FC31
:1018500007C0621773078407950721F008F4009406
:101860000794989408959A95BB0F661F771F881F59
:1018700011249923A1F08823B2F79F3F59F0BB0FA1
:1018800048F421F4002011F460FF04C06F5F7F4F23
:101890008F4F9F4F881F9795879597F908952CC074
:1018A0009FEF80EC0895052E092607FA440F551F77
:1018B0005F3F79F0AA27A51708F051E04795880FF8
:1018C000991F9F3F31F0BB27B91708F091E087952A
:1018D00008959F919F911124E3CF97FB880F991F43
:1018E0009F3F31F0BB27B91708F091E08795089525
:1018F0009F919F911124D4CF662777278827992716
:101900000895D1DF01D0B4CF992339F0552329F0C0
:101910009F575F57950F13F4CAF1F1CF91589F3F2E
:10192000E1F3A62F00241124BB2766275527F8E0F2
:10193000A69520F4020E131EB41F651F220F331F3D
:10194000441F551FFA95A1F7F8E0E72F7727F8E035
:10195000E69520F4130EB41F651F7A1F330F441F42
:10196000551FAA1FFA95A1F7F82F8827F69520F49E
:10197000B40F651F7A1F8E1F440F551FAA1FEE1F3D
:10198000FF23A1F788231AF4939539F489CF000C2B
:10199000111CBB1F661F771F881F0128089509D0DF
:1019A00001921A94E1F7089501900BD01A94E1F78F
:1019B0000895E199FECFBFBBAEBBE09A11960DB280
:1019C0000895E199FECFBFBBAEBB0DBA11960FB61D
:1019D000F894E29AE19A0FBE0895AA1BBB1B51E14D
:1019E00007C0AA1FBB1FA617B70710F0A61BB70B8F
:1019F000881F991F5A95A9F780959095682F792F80
:081A00008A2F9B2F0895FFCFF0
:00000001FF
